:100000004AC064C063C05DC6D1C53EC603C61FC634
:10001000B0C568C55BC0AFC659C0E2C615C156C001
:1000200055C054C053C0084AD73B3BCE016E84BC78
:10003000BFFDC12F3D6C74319ABD56833DDA3D0042
:10004000C77F11BED9E4BB4C3E916BAAAABE00008B
:1000500000803F583A256420593A25642066693A61
:1000600025642E2564200D0A0030313233343536B4
:10007000373839414243444546000000010008003A
:1000800040000001000400000100080020004000C2
:1000900080000001000411241FBECFE5D4E0DEBFC4
:1000A000CDBF11E0A0E6B0E0EAEDFCE102C00590B2
:1000B0000D92A836B107D9F712E0A8E6B1E001C069
:1000C0001D92AA3DB107E1F702D005CE99CF9F92CC
:1000D000AF92BF92CF92DF92EF92FF920F931F9356
:1000E000CF93DF93EBD660E875E280E090E00BD62B
:1000F00083EA96E060D139D360D014BA15BA87E0AC
:100100006FD080E072D0CC24DD2410E0C0E0D0E0DD
:1001100033E5A32E30E0B32E9924939409C080E0F8
:1001200079D0C80FD91F81E075D0C80ED91E1F5FC6
:100130001032A8F3CE0160E270E0E3DAEB01C050C8
:10014000D240C60160E270E0DCDAC12C2EEFD22E84
:10015000C60ED71EBE01882777FD8095982F5FD8E1
:100160007B018C01B601882777FD8095982F57D8A1
:10017000A80197015CDB20E030E044E353E4B5D60E
:100180002BED3FE049E450E4A5D70ADC1F921F9213
:10019000A0D87F936F93DF92CF92DF93CF93BF92DC
:1001A000AF929F9254D210E08DB79EB70B960FB6C8
:1001B000F8949EBF0FBE8DBFB2CF379A359886B1E7
:1001C000887F866086B987B18F73806487B93D98D0
:1001D000339A1092B9027894089533983798089515
:1001E00096B1987F982B96B9089597B18295880F0C
:1001F000880F807C9F73982B97B9089597B18F7162
:10020000907E892B87B90895349A369A089586B1DD
:10021000807408951092B90297B18F71907E892BE6
:1002200087B9349A369A3699FECF24B145B1942FC6
:1002300080E030E0282B392BC9010895EBDF96953B
:1002400087959695879508951F920F920FB60F92F6
:1002500011248F938FEF8093B9028F910F900FBE6F
:100260000F901F901895FC018FB7F89471836083ED
:100270005383428317821682158214828FBF08959A
:10028000CF93DF93DC014FB7F894EC018C819D8113
:10029000892B11F4E0E01CC0FD0186819781ED916E
:1002A000FC911197E80FF91FE0810196ED019F8302
:1002B0008E832A813B818217930720F0821B930B48
:1002C0009F838E83ED018C819D8101979D838C831B
:1002D0004FBF8E2FDF91CF910895FC014FB7F89457
:1002E0008481958168177907B0F486819781860F9C
:1002F000971F97838683228133818217930720F08B
:10030000821B930B9783868384819581861B970B31
:100310009583848302C0158214824FBF0895FC0127
:10032000CB012FB7F8942FBF26813781628173816B
:10033000820F931FD2D90190F081E02DE80FF91FB1
:10034000808108951F93CF93DF93EC01162F4FB751
:10035000F8942C813D816A817B812617370790F4C0
:100360008E819F81820F931FB8D9E881F981E80FB0
:10037000F91F10838C819D8101969D838C834FBFD3
:100380008FEF02C04FBF80E0DF91CF911F910895A2
:10039000FC018FB7F8948FBF2281338184819581CE
:1003A000281B390BC9010895FC018FB7F8941582F9
:1003B00014828FBF08959093690180936801089516
:1003C0001F93182F8A3031F4E0916801F091690190
:1003D0008DE00995E0916801F0916901812F0995FF
:1003E0001F910895CF93DF93EC01009719F405C096
:1003F0002196E6DF88818823D9F7DF91CF91089590
:10040000EF92FF920F931F93CF93DF938C017A01AA
:100410000097E1F020E030E02617370738F4F801C4
:1004200081918F012F5F3F4F8823B1F7C0E0D0E06B
:100430000AC0F8018081882319F00F5F1F4F01C0A7
:1004400080E2BEDF2196CE15DF0598F3DF91CF91D4
:100450001F910F91FF90EF900895CF93DF93EC01E0
:10046000009711F406C0ACDFFE0121968491882329
:10047000D1F7DF91CF9108958AE0A2DF0895E82FA8
:10048000F0E0EF70F070E759FF4FE4918E2F98DFA6
:1004900008951F93182F82958F70F1DF812FEFDF62
:1004A0001F9108951F93182F892FF3DF812FF1DFFC
:1004B0001F910895EF92FF920F931F937B018C0180
:1004C000C801AA27BB27EEDFC701ECDF1F910F9100
:1004D000FF90EF9008952F923F924F925F926F920C
:1004E0007F928F929F92AF92BF92CF92DF92EF92C4
:1004F000FF920F931F93DF93CF93CDB7DEB7A397F0
:100500000FB6F894DEBF0FBECDBF4AA32BA33701B1
:100510004801442351F017FF08C0EE24FF2487014F
:10052000E618F7080809190902C084017301262E8C
:10053000262F215090E03AA1311191E0291B29A3E7
:1005400018A2A82EBB24A7FCB094CB2CDB2CC8018E
:10055000B701A6019501E8D8FB01EF70F070E759EB
:10056000FF4F64916F8FC801B701A6019501DCD8D8
:10057000C901DA017C018D019EE1492E512C4C0EFE
:100580005D1E39A023C0E114F10401051105B9F085
:10059000C801B701A6019501C7D8FB01EF70F07043
:1005A000E759FF4F6491F2016083C801B701A601CA
:1005B0009501BAD8C901DA017C018D0103C02BA1D4
:1005C000F20120833A940894410851083320D9F667
:1005D000CE014F968C0139A1031B11098AA18823F2
:1005E000D9F097FE05C08DE2F80182938F0114C007
:1005F000C8010197611471048104910419F08C0100
:100600008BE202C08C0180E2F801808305C0F80112
:1006100081918F01D5DE2A942220C9F7A3960FB6C7
:10062000F894DEBF0FBECDBFCF91DF911F910F9128
:10063000FF90EF90DF90CF90BF90AF909F908F9002
:100640007F906F905F904F903F902F9008957F9292
:100650008F929F92AF92BF92CF92DF92EF92FF92D2
:100660000F931F93DF93CF93CDB7DEB77888C988F8
:10067000DA8853E1E52EF12CEC0EFD1E13C0882321
:1006800081F480E090E0CF91DF911F910F91FF9076
:10069000EF90DF90CF90BF90AF909F908F907F9022
:1006A00008958EDE96012F5F3F4F772021F0F601EF
:1006B0006901849103C0F601808169018532F9F6F0
:1006C0002F5F3F4F772021F0F6016901849103C02D
:1006D000F60180816901843629F0883781F08336FC
:1006E00001F706C000E117E24AE0A42EB12C0CC0CD
:1006F000F701808122E030E0E20EF31ED2CF00E06D
:1007000010E130E1A32EB12C22E0822E912C8E0C30
:100710009F1CF701E080F1808436A1F4F7FE0FC042
:10072000F094E194F108F3948DE24ADE08C0C80128
:100730006AE070E0D2D78B016230710518F0E016E4
:10074000F106A8F3C701B801C8D7862F98DEC70104
:10075000B801C3D77C01C801B501BFD78B016115B2
:10076000710581F774019ECF089580E090E0FC014F
:10077000EE0FFF1FE659FE4F11821082019687305F
:100780009105A9F783B7887F826083BF12BE89B7BE
:10079000816089BF1092BA021092BB021092BC0213
:1007A0001092BD028EB5887F83608EBD1DBC1CBCBF
:1007B00089B7846089BF85B5887F846085BD14BC96
:1007C00089B7806489BF1092C2021092C30210924E
:1007D000C4021092C5027894089583B7887F82601E
:1007E00083BF12BE89B7816089BF1092BA0210928E
:1007F000BB021092BC021092BD0208958EB5887F94
:1008000083608EBD1DBC1CBC89B7846089BF089500
:1008100085B5887F846085BD14BC89B7806489BF35
:100820001092C2021092C3021092C4021092C5022A
:10083000089593B7987F982B93BF08959EB5987F9E
:10084000982B9EBD089595B5987F982B95BD0895DA
:1008500083B7E82FF0E0E770F070EE0FFF1FE65867
:10086000FF4F25913491C90108958EB5E82FF0E02E
:10087000E770F070EE0FFF1FE658FF4F259134919F
:10088000C901089585B5E82FF0E0E770F070EE0F2C
:10089000FF1FEA57FF4F25913491C9010895873012
:1008A00040F4E82FF0E0EE0FFF1FE659FE4F718392
:1008B00060830895873040F4E82FF0E0EE0FFF1FCB
:1008C000E659FE4F118210820895EF92FF920F9326
:1008D0001F93CF93DF93EC0112B71092BE021092D8
:1008E000BF021092C0021092C10283B7E82FF0E05D
:1008F000E770F070EE0FFF1FE658FF4F259134911F
:1009000040E050E060E072E18AE790E02FD7B90163
:10091000CA01693B2DE8720726E0820720E09207B2
:1009200090F437E2C131D30770F49E0140E050E00B
:10093000B5D628EE33E040E050E0F6D6C901DA0142
:10094000BC01CD011FC028EE33E040E050E0ECD602
:10095000CA01B9019E0140E050E0A0D613C08091C9
:10096000BE029091BF02A091C002B091C10285B7B2
:100970008F7885BF85B7806885BF889585B78F7765
:1009800085BF08C09B01AC01210F311D411D511DC8
:1009900079018A012091BE023091BF024091C002CC
:1009A0005091C10282B790E0A0E0B0E0542F432FF5
:1009B000322F2227822B932BA42BB52B8E159F052C
:1009C000A007B10760F2DF91CF911F910F91FF90C7
:1009D000EF9008951092BA021092BB021092BC02DE
:1009E0001092BD0208952091BA023091BB0240914D
:1009F000BC025091BD02B901CA0108951092C20211
:100A00001092C3021092C4021092C5020895209160
:100A1000C2023091C3024091C4025091C502B90193
:100A2000CA010895893031F48FB582608FBD8FB5CA
:100A30008E7F0AC08A3019F48FB5826002C08FB5EC
:100A40008D7F8FBD8FB581608FBD1BBC1ABC19BC5B
:100A500018BC08952FB52E7F2FBD2FB522602FBD56
:100A60002EB528602EBD2EB520612EBD97BD86BD4A
:100A70001BBC1ABC19BC18BC08958FB58D7F8FBDE7
:100A80008FB58E7F8FBD8FB58F778FBD8FB58F7BE5
:100A90008FBD8FB58F7D8FBD8FB58F7E8FBD089534
:100AA0008FB580688FBD8FB58F7B8FBD08958FB553
:100AB00080628FBD8FB58F7E8FBD08958FB58F7784
:100AC0008FBD8FB58F7B8FBD08958FB58F7D8FBD07
:100AD0008FB58F7E8FBD08959BBD8ABD089599BD4A
:100AE00088BD08951F920F920FB60F9211248F9315
:100AF0009F93AF93BF93EF93FF938091BA0290912E
:100B0000BB02A091BC02B091BD020196A11DB11D16
:100B10008093BA029093BB02A093BC02B093BD0233
:100B20008091BE029091BF02A091C002B091C1021B
:100B30000196A11DB11D8093BE029093BF02A093A8
:100B4000C002B093C10280916A0190916B01892B20
:100B500029F0E0916A01F0916B010995FF91EF9105
:100B6000BF91AF919F918F910F900FBE0F901F90EB
:100B700018951F920F920FB60F9211248F939F9387
:100B8000EF93FF9380916C0190916D01892B29F077
:100B9000E0916C01F0916D010995FF91EF919F91AA
:100BA0008F910F900FBE0F901F9018951F920F926C
:100BB0000FB60F9211248F939F93AF93BF93EF9330
:100BC000FF938091C2029091C302A091C402B091A0
:100BD000C5020196A11DB11D8093C2029093C3026C
:100BE000A093C402B093C5028091740190917501E5
:100BF000892B29F0E0917401F09175010995FF911D
:100C0000EF91BF91AF919F918F910F900FBE0F9079
:100C10001F9018951F920F920FB60F9211248F9369
:100C20009F93EF93FF9380916E0190916F01892BB9
:100C300029F0E0916E01F0916F010995FF91EF911C
:100C40009F918F910F900FBE0F901F9018951F923C
:100C50000F920FB60F9211248F939F93EF93FF93F0
:100C60008091700190917101892B29F0E0917001C0
:100C7000F09171010995FF91EF919F918F910F90E4
:100C80000FBE0F901F9018951F920F920FB60F92E4
:100C900011248F939F93EF93FF9380917201909112
:100CA0007301892B29F0E0917201F091730109958C
:100CB000FF91EF919F918F910F900FBE0F901F901A
:100CC00018951F920F920FB60F9211248F939F9336
:100CD000EF93FF938091760190917701892B29F012
:100CE000E0917601F09177010995FF91EF919F9145
:100CF0008F910F900FBE0F901F9018959093B80290
:100D00008093B70208959B01AC01605C7D4B804FDE
:100D10009F4FF3E0660F771F881F991FFA95D1F751
:100D2000E4E0220F331F441F551FEA95D1F7FCD48E
:100D30002150304029B930BD089587EC92E00895E4
:100D400080ED92E00895982F8091C6028823E1F308
:100D50009CB91092C60208951092CC021092CB0258
:100D600008958091CB029091CC02892B11F080E004
:100D700008958FEF08951F920F920FB60F921124CE
:100D80006F938F939F93EF93FF936CB18091B70212
:100D90009091B802892B39F0E091B702F091B80236
:100DA000862F09950EC087EC92E0CCDA882349F4AF
:100DB0008091D8029091D90201969093D9028093A4
:100DC000D802FF91EF919F918F916F910F900FBE7D
:100DD0000F901F901895682F80ED92E0B3DA089578
:100DE0001F920F920FB60F9211248F939F938091B1
:100DF000CF02882369F08091D4029091D502892B8B
:100E000029F080ED92E03CDA8CB905C01092CF0257
:100E10008FEF8093C6029F918F910F900FBE0F901E
:100E20001F9018958FEF8093CF0280ED92E028DA23
:100E3000982F8091C6028823E1F39CB91092C602D4
:100E40000895CF93DF93EC018091C9029091CA027B
:100E5000892B61F08091CB029091CC02892B31F0EB
:100E600087EC92E00DDA88838FEF01C080E0DF919C
:100E7000CF910895DF93CF930F92CDB7DEB7CE0118
:100E80000196DFDF882319F42FEF3FEF03C089813C
:100E9000282F30E0C9010F90CF91DF9108954FEFD7
:100EA00050E068E771E087EC92E0DDD940E450E083
:100EB00067E772E080ED92E0D6D90895F0DF1092F6
:100EC000B8021092B70288ED8AB960E875E280E056
:100ED00090E019DF8FEF8093C6021092CF0210923C
:100EE000D9021092D80278940895A0E2B0E0EAE71F
:100EF000F7E057C469837A838B839C832D833E8379
:100F00004F835887BE01675F7F4FCE01019656D34E
:100F1000BE016F5E7F4FCE01059650D3998592300A
:100F200088F089898230C8F0943019F4823051F405
:100F300004C0843029F4923081F480E690E0C6C089
:100F4000923049F420E09A858A89981321E02A8713
:100F5000CE010996BBC0823049F420E09A858A8987
:100F6000981321E02A8BCE014196B0C02D843E8497
:100F70004F8458886D887E888F88988CEE24FF2453
:100F80008701AA24BB24650140E050E060E070E0E6
:100F9000E0E0F0E0C10181709070892BE9F0E60C8F
:100FA000F71C081D191D9A01AB012A0D3B1D4C1D94
:100FB0005D1D80E090E0A0E0B0E0E614F7040805D5
:100FC000190520F481E090E0A0E0B0E0BA01A901A9
:100FD000480F591F6A1F7B1FAA0CBB1CCC1CDD1CB1
:100FE00097FE08C081E090E0A0E0B0E0A82AB92A0E
:100FF000CA2ADB2A3196E032F10549F0660C771CEB
:10100000881C991C5694479437942794C3CFFA852B
:10101000EA892B893C898B859C85280F391F2E5F97
:101020003F4F17C0CA0181709070892B61F01695EF
:101030000795F794E79480E090E0A0E0B0E8E82A14
:10104000F92A0A2B1B2B76956795579547952F5FA5
:101050003F4F77FDE7CF0CC0440F551F661F771F2A
:1010600017FD4160EE0CFF1C001F111F2150304086
:10107000403090E0590790E0690790E4790760F309
:101080002B8F3C8FDB01CA018F779070A070B070FE
:1010900080349105A105B10561F447FD0AC0E11452
:1010A000F1040105110529F0405C5F4F6F4F7F4F40
:1010B00040781A8EFE1711F081E08A8F4D8F5E8F77
:1010C0006F8F78A383E0898FCE014996A2D1A09635
:1010D000E2E183C3A8E1B0E0EFE6F8E06AC3698328
:1010E0007A838B839C832D833E834F835887B9E01B
:1010F000EB2EF12CEC0EFD1EB701CE0101965ED257
:101100008E010F5E1F4FB801CE01059657D229857B
:10111000223008F47CC03989323010F4B8017AC02A
:101120008A859A8989278A87243011F0223031F400
:10113000231709F06CC060E670E06CC0343039F4FD
:101140001D861E861F86188A1C861B8604C03230A8
:1011500021F484E08987B7015DC02B853C858B89AC
:101160009C89281B390B3C872B87ED84FE840F85D7
:101170001889AD88BE88CF88D88CEA14FB040C058A
:101180001D0540F4EE0CFF1C001F111F21503040C4
:101190003C872B8720E030E040E050E080E090E0AA
:1011A000A0E0B0E46FE170E0EA14FB040C051D055B
:1011B00040F0282B392B4A2B5B2BEA18FB080C0933
:1011C0001D09B695A79597958795EE0CFF1C001FF6
:1011D000111F6150704041F7DA01C9018F7790709B
:1011E000A070B07080349105A105B10561F427FDB0
:1011F0000AC0E114F1040105110529F0205C3F4FFC
:101200004F4F5F4F20782D873E874F87588BBE0109
:10121000675F7F4FCB01FDD06896EAE0E6C2A8E0A9
:10122000B0E0E4E1F9E0C6C29B01AC0183E0898350
:10123000DA01C9018827B7FD83959927AA27BB271B
:10124000B82E211531054105510519F482E0898335
:1012500039C08823A9F0203080E0380780E04807B3
:1012600080E8580729F460E070E080E09FEC2EC031
:10127000EE24FF248701E21AF30A040B150B02C0C7
:1012800079018A018EE1C82ED12CDC82CB82ED82DD
:10129000FE820F831887C801B7016CD0019718161A
:1012A000190684F4082E04C0EE0CFF1C001F111F49
:1012B0000A94D2F7ED82FE820F831887C81AD90AE2
:1012C000DC82CB82BA82CE010196A3D02896E9E0D7
:1012D0008DC2ACE0B0E0EEE6F9E073C269837A83D8
:1012E0008B839C83BE016B5F7F4FCE01019666D1DD
:1012F0008D81823061F1823050F1843021F48E8111
:10130000882351F12EC02F81388537FD20C06E8192
:101310002F3131051CF06623F9F023C08EE190E0F7
:10132000821B930B29853A854B855C8504C05695B5
:101330004795379527958A95D2F76623B1F0509552
:101340004095309521953F4F4F4F5F4F0EC020E0A5
:1013500030E040E050E009C02FEF3FEF4FEF5FE794
:1013600004C020E030E040E050E8B901CA012C960A
:10137000E2E043C2EF92FF920F931F937B018C0137
:1013800080E0E81680E0F80681E0080780E01807B2
:1013900088F48FEFE816F1040105110531F028F00B
:1013A00088E090E0A0E0B0E017C080E090E0A0E02E
:1013B000B0E012C080E0E81680E0F80680E00807A0
:1013C00081E0180728F088E190E0A0E0B0E004C0D8
:1013D00080E190E0A0E0B0E020E230E040E050E0CA
:1013E000281B390B4A0B5B0B04C016950795F79425
:1013F000E7948A95D2F7F701E859FF4F8081281BBF
:10140000310941095109C9011F910F91FF90EF90D6
:101410000895DF92EF92FF920F931F93FC01E480F7
:10142000F58006811781D1808081823048F480E088
:1014300090E0A0E1B0E0E82AF92A0A2B1B2BA5C016
:10144000843009F49FC0823021F4EE24FF24870108
:1014500005C0E114F1040105110519F4E0E0F0E024
:1014600096C0628173819FEF623879070CF05BC090
:1014700022E83FEF261B370B2A3131052CF020E004
:1014800030E040E050E02AC0B801A701022E04C0BD
:1014900076956795579547950A94D2F781E090E045
:1014A000A0E0B0E004C0880F991FAA1FBB1F2A95B7
:1014B000D2F70197A109B1098E219F21A023B12361
:1014C0000097A105B10521F081E090E0A0E0B0E037
:1014D0009A01AB01282B392B4A2B5B2BDA01C9016E
:1014E0008F779070A070B07080349105A105B10520
:1014F00039F427FF09C0205C3F4F4F4F5F4F04C0B6
:10150000215C3F4F4F4F5F4FE0E0F0E02030A0E024
:101510003A07A0E04A07A0E45A0710F0E1E0F0E043
:1015200079018A0127C06038710564F5FB01E15833
:10153000FF4FD801C7018F779070A070B0708034D2
:101540009105A105B10539F4E7FE0DC080E490E0F6
:10155000A0E0B0E004C08FE390E0A0E0B0E0E80ECF
:10156000F91E0A1F1B1F17FF05C016950795F79454
:10157000E794319687E016950795F794E7948A9556
:10158000D1F705C0EE24FF248701EFEFF0E06E2FC6
:10159000679566276795902F9F77D794DD24D7941A
:1015A0008E2F8695492F462B582F5D29B701CA01EA
:1015B0001F910F91FF90EF90DF900895FC01DB01E8
:1015C000408151812281622F6F7770E0221F222794
:1015D000221F9381892F880F822B282F30E0991F9B
:1015E0009927991FFD0191832115310581F5411539
:1015F00051056105710511F482E032C082E89FEF68
:10160000FD01938382839A01AB0167E0220F331FB0
:10161000441F551F6A95D1F783E08C930AC0220FAF
:10162000331F441F551FFD018281938101979383CE
:1016300082832030F0E03F07F0E04F07F0E45F07DF
:1016400070F3FD01248335834683578308952F3F2C
:10165000310581F4411551056105710519F484E0E6
:101660008C93089564FF03C081E08C9301C01C92A9
:10167000FD010FC02F573040FD013383228383E0EB
:101680008C9387E0440F551F661F771F8A95D1F70B
:10169000706444835583668377830895629FD00185
:1016A000739FF001829FE00DF11D649FE00DF11D1D
:1016B000929FF00D839FF00D749FF00D659FF00DCC
:1016C0009927729FB00DE11DF91F639FB00DE11DB9
:1016D000F91FBD01CF0111240895AA1BBB1B51E1C5
:1016E00007C0AA1FBB1FA617B70710F0A61BB70B92
:1016F000881F991F5A95A9F780959095BC01CD0137
:10170000089597FB092E07260AD077FD04D0E5DF60
:1017100006D000201AF4709561957F4F0895F6F772
:10172000909581959F4F0895A1E21A2EAA1BBB1B8D
:10173000FD010DC0AA1FBB1FEE1FFF1FA217B3079D
:10174000E407F50720F0A21BB30BE40BF50B661FB3
:10175000771F881F991F1A9469F760957095809577
:1017600090959B01AC01BD01CF01089597FB092E17
:1017700005260ED057FD04D0D7DF0AD0001C38F460
:1017800050954095309521953F4F4F4F5F4F0895AD
:10179000F6F790958095709561957F4F8F4F9F4F8D
:1017A00008952F923F924F925F926F927F928F9205
:1017B0009F92AF92BF92CF92DF92EF92FF920F93E0
:1017C0001F93CF93DF93CDB7DEB7CA1BDB0B0FB6EA
:1017D000F894DEBF0FBECDBF09942A8839884888A7
:1017E0005F846E847D848C849B84AA84B984C8843D
:1017F000DF80EE80FD800C811B81AA81B981CE0F34
:10180000D11D0FB6F894DEBF0FBECDBFED01089518
:1018100033D158F080E891E009F49EEF34D128F0FC
:1018200040E851E059F45EEF09C0FEC07DC1E92FE8
:10183000E07841D168F3092E052AC1F3261737074E
:101840004807590738F00E2E07F8E02569F0E02523
:10185000E0640AC0EF6307F8009407FADB01B901FE
:101860009D01DC01CA01AD01EF9341D013D10AD033
:101870005F91552331F02BED3FE049E450FD49ECF9
:10188000C6C10895DF93DD27B92FBF7740E85FE336
:101890001616170648075B0710F4D92F4CD19F93F3
:1018A0008F937F936F93AFD1E6E2F0E0C0D0F2D098
:1018B0002F913F914F915F914FD1DD2349F0905887
:1018C000A2EA2AED3FE049EC5FE3D0785D27B0D192
:1018D000DF91E0C0D8D040F0CFD030F021F45F3FAE
:1018E00019F071C0511121C19FC0E5D098F399231F
:1018F000C9F35523B1F3951B550BBB27AA276217D4
:101900007307840738F09F5F5F4F220F331F441F18
:10191000AA1FA9F333D00E2E3AF0E0E830D0915050
:101920005040E695001CCAF729D0FE2F27D0660F3D
:10193000771F881FBB1F261737074807AB07B0E87C
:1019400009F0BB0B802DBF01FF2793585F4F2AF092
:101950009E3F510568F037C0E8C05F3FECF3983E0A
:10196000DCF3869577956795B795F7959F5FC9F7EF
:10197000880F911D9695879597F90895E1E0660F78
:10198000771F881FBB1F621773078407BA0720F0F1
:10199000621B730B840BBA0BEE1F88F7E09508955A
:1019A000ACD080F09F3740F491110EF0BEC060E0E3
:1019B00070E080E89FEB089526F41B16611D711DF1
:1019C000811D07C021C097F99F6780E870E060E043
:1019D0000895882371F4772321F09850872B762F70
:1019E00007C0662311F499270DC09051862B70E033
:1019F00060E02AF09A95660F771F881FDAF7880F44
:101A00009695879597F908959F3F49F0915028F44E
:101A1000869577956795B7959F5F80389F4F880F1C
:101A20009695879597F908959FEF80EC0895DF9339
:101A3000CF931F930F93FF92EF92DF927B018C0164
:101A4000689405C0DA2EEF0187D0FE01E894A591D5
:101A50002591359145915591AEF3EF01E9D0FE0105
:101A60009701A801DA9479F7DF90EF90FF900F913A
:101A70001F91CF91DF91089500240A94161617063E
:101A800018060906089500240A941216130614066F
:101A900005060895092E0394000C11F4882352F0D2
:101AA000BB0F40F4BF2B11F460FF04C06F5F7F4F8A
:101AB0008F4F9F4F089557FD9058440F551F59F071
:101AC0005F3F71F04795880F97FB991F61F09F3F2B
:101AD00079F087950895121613061406551FF2CF54
:101AE0004695F1DF08C0161617061806991FF1CFA4
:101AF00086957105610508940895E5DFA0F0BEE7BD
:101B0000B91788F4BB279F3860F41616B11D672FEC
:101B1000782F8827985FF7CF869577956795B11DC1
:101B200093959639C8F30895E894BB2766277727DD
:101B3000CB0197F908959B01AC0160E070E080E86B
:101B40009FE3C8CA99DF28F09EDF18F0952309F0BB
:101B50003ACF6ACF1124E9CFAEDFA0F3959FD1F33E
:101B6000950F50E0551F629FF001729FBB27F00D4B
:101B7000B11D639FAA27F00DB11DAA1F649F6627A0
:101B8000B00DA11D661F829F2227B00DA11D621FEF
:101B9000739FB00DA11D621F839FA00D611D221FA9
:101BA000749F3327A00D611D231F849F600D211D8D
:101BB000822F762F6A2F11249F5750408AF0E1F030
:101BC00088234AF0EE0FFF1FBB1F661F771F881F79
:101BD00091505040A9F79E3F510570F0F4CEA5CF2B
:101BE0005F3FECF3983EDCF3869577956795B79564
:101BF000F795E7959F5FC1F7FE2B880F911D96958E
:101C0000879597F908959B01AC016FC95058BB2780
:101C1000AA270ED03FCF30DF30F035DF20F031F48F
:101C20009F3F11F41EF400CF0EF4E095E7FBCBCEFE
:101C3000E92F41DF80F3BA1762077307840795071E
:101C400018F071F49EF570CF0EF4E0950B2EBA2FBC
:101C5000A02D0B01B90190010C01CA01A0011124B2
:101C6000FF27591B99F0593F50F4503E68F11A165E
:101C7000F040A22F232F342F4427585FF3CF4695EF
:101C800037952795A795F0405395C9F77EF41F1611
:101C9000BA0B620B730B840BBAF09150A1F0FF0FDB
:101CA000BB1F661F771F881FC2F70EC0BA0F621FC7
:101CB000731F841F48F4879577956795B795F795B7
:101CC0009E3F08F0B3CF9395880F08F09927EE0F49
:0A1CD000979587950895F894FFCFCB
:101CDA0000000000000000000001020203030303E9
:101CEA0004040404040404040505050505050505A2
:101CFA000505050505050505060606060606060682
:101D0A000606060606060606060606060606060669
:101D1A000606060606060606070707070707070751
:101D2A000707070707070707070707070707070739
:101D3A000707070707070707070707070707070729
:101D4A000707070707070707070707070707070719
:101D5A000707070707070707080808080808080801
:101D6A0008080808080808080808080808080808E9
:101D7A0008080808080808080808080808080808D9
:101D8A0008080808080808080808080808080808C9
:101D9A0008080808080808080808080808080808B9
:101DAA0008080808080808080808080808080808A9
:101DBA000808080808080808080808080808080899
:101DCA000808080808080808080808080808080889
:081DDA000808080808080808C1
:00000001FF
